:100000000C9446000C9465000C9465000C946500FB
:100010000C9465000C9465000C9465000C946500CC
:100020000C9465000C9465000C9465000C946500BC
:100030000C9465000C9465000C9465000C946500AC
:100040000C9465000C9465000C9465000C9465009C
:100050000C9465000C9465000C9465000C9465008C
:100060000C9465000C9465000C9465000C9465007C
:100070000C9465000C9465000C9465000C9465006C
:100080000C9465000C9465000C94650011241FBE4F
:10009000CFEFD0E1DEBFCDBF11E0A0E0B1E0E8ECF2
:1000A000FCE000E00BBF02C007900D92A433B10743
:1000B000D9F711E0A4E3B1E001C01D92AD34B1075E
:1000C000E1F70E9411030C9463060C940000CF9397
:1000D000DF93CDB7DEB722970FB6F894DEBF0FBE21
:1000E000CDBF9A83898305C089819A8101979A83BC
:1000F000898389819A810097B9F722960FB6F8947F
:10010000DEBF0FBECDBFDF91CF910895CF93DF93B8
:10011000CDB7DEB7A5E3B0E0E5E3F0E08081846031
:100120008C9388E795E00E946700A5E3B0E0E5E3E3
:10013000F0E090818BEF89238C93DF91CF9108952C
:10014000CF93DF93CDB7DEB7A5E3B0E0E5E3F0E012
:1001500090818EEF89238C9380E197E20E94670063
:10016000E5E3F0E080E380830E94860088EE93E080
:100170000E946700E5E3F0E080E380830E94860050
:1001800088EE93E00E946700E5E3F0E080E380837F
:100190000E94860088EE93E00E946700E5E3F0E0AD
:1001A00080E280830E948600DF91CF910895CF93F3
:1001B000DF93CDB7DEB721970FB6F894DEBF0FBE41
:1001C000CDBF898389818F6080933C01A5E3B0E036
:1001D000E5E3F0E08081982F906F80913C018923C6
:1001E0008C93A5E3B0E0E5E3F0E090818EEF892306
:1001F0008C930E94860089818295807F80933C0148
:10020000A5E3B0E0E5E3F0E08081982F9F70809156
:100210003C01892B8C93A5E3B0E0E5E3F0E090810D
:100220008EEF89238C930E94860021960FB6F89456
:10023000DEBF0FBECDBFDF91CF910895CF93DF9387
:10024000CDB7DEB721970FB6F894DEBF0FBECDBF96
:10025000898389818F6080933C01A5E3B0E0E5E369
:10026000F0E08081982F906F80913C0189238C93DE
:10027000A5E3B0E0E5E3F0E0808181608C930E942B
:10028000860089818295807F80933C01A5E3B0E060
:10029000E5E3F0E08081982F9F7080913C01892BED
:1002A0008C93A5E3B0E0E5E3F0E0808181608C937E
:1002B0000E94860021960FB6F894DEBF0FBECDBF18
:1002C000DF91CF910895CF93DF93CDB7DEB7249719
:1002D0000FB6F894DEBF0FBECDBF9C838B831A820E
:1002E000198210C089819A819C018B819C81F901BE
:1002F000E80FF91F80810E941E0189819A81019671
:100300009A83898329813A818B819C81DC01FD015B
:1003100001900020E9F73197CF018A1B9B0B28172A
:10032000390700F324960FB6F894DEBF0FBECDBF99
:10033000DF91CF9108950F931F93CF93DF93CDB7A4
:10034000DEB7AE970FB6F894DEBF0FBECDBF6BA77A
:100350007CA78DA79EA71A8219828BA59CA5ADA507
:10036000BEA5BB2394F48DE20E941E018BA59CA523
:10037000ADA5BEA5B095A095909581959F4FAF4F27
:10038000BF4F8BA79CA7ADA7BEA78A818F5F8A832B
:100390008A81082F11278BA59CA5ADA5BEA52AE0B3
:1003A00030E040E050E0BC01CD010E941206DC01CB
:1003B000CB01AC019801220F331FCE010196820FB1
:1003C000931FFC013296518340838BA59CA5ADA55C
:1003D000BEA52AE030E040E050E0BC01CD010E9423
:1003E0001206DA01C9018BA79CA7ADA7BEA78BA5F2
:1003F0009CA5ADA5BEA50097A105B10531F68A81E2
:10040000898389818A8313C08A8199279C01220F5D
:10041000331FCE010196820F931FFC01329680811B
:100420009181805D0E941E018A8181508A838A8128
:10043000882351F7AE960FB6F894DEBF0FBECDBF3E
:10044000DF91CF911F910F910895CF93DF93CDB797
:10045000DEB726970FB6F894DEBF0FBECDBF9E83E2
:100460008D831C821B821A8219828D819E812AE0D3
:1004700030E0B9010E94FF059A8389838D819E81B6
:100480002AE030E0B9010E94FF05CB019C838B83F9
:100490008B81805D0E941E018981805D0E941E010A
:1004A00026960FB6F894DEBF0FBECDBFDF91CF9179
:1004B0000895CF93DF93CDB7DEB722970FB6F894A8
:1004C000DEBF0FBECDBF1A82198208C080E80E942D
:1004D000D70089819A8101969A83898389819A813B
:1004E000181619069CF722960FB6F894DEBF0FBEB9
:1004F000CDBFDF91CF910895CF93DF93CDB7DEB716
:1005000022970FB6F894DEBF0FBECDBF1A821982B4
:1005100008C080EC0E94D70089819A8101969A8355
:10052000898389819A81883291059CF322960FB63E
:10053000F894DEBF0FBECDBFDF91CF910895CF936A
:10054000DF93CDB7DEB722970FB6F894DEBF0FBEAC
:10055000CDBF9A83898389819A818130910571F415
:10056000A5E3B0E0E5E3F0E0808180628C93A4E352
:10057000B0E0E5E3F0E0808180628C9389819A812C
:10058000009781F4A5E3B0E0E5E3F0E090818FED22
:1005900089238C93A4E3B0E0E4E3F0E090818FED55
:1005A00089238C9322960FB6F894DEBF0FBECDBF81
:1005B000DF91CF910895CF93DF93CDB7DEB7EBE313
:1005C000F0E01082EAE3F0E080E48083E8E3F0E02A
:1005D0001082E7E3F0E01082E5E3F0E01082E4E36C
:1005E000F0E087EF8083E2E3F0E080EC8083E1E3FA
:1005F000F0E088E08083E3E2F0E01082E2E2F0E005
:1006000080E38083E2E6F0E01082E1E6F0E0108231
:10061000E5E6F0E01082E4E6F0E01082DF91CF91B1
:100620000895CF93DF93CDB7DEB76A970FB6F894EE
:10063000DEBF0FBECDBF0E94DB020E94A00088E09B
:100640000E94D70000C0E9E3F0E080819927817023
:1006500090701F861E86009721F421E030E03F87CE
:100660002E878091000190910101EE85FF85E8239E
:10067000F923FD87EC8780913501909136011B8627
:100680001A86009721F421E030E03B872A878C8589
:100690009D85EA85FB858E239F230097A1F08CE042
:1006A0000E94D70081E00E94D70082E091E00E9482
:1006B0006301109201011092000181E090E090939B
:1006C000360180933501E9E3F0E08081992782705B
:1006D000907019861886009721F421E030E0398760
:1006E0002887809100019091010128853985282370
:1006F000392380913501909136018223932300970D
:1007000009F493C081E00E94D70080E80E94D700DE
:1007100010923B0110923A0111C080913A019091E0
:100720003B01FC01E35CFE4F108280913A01909105
:100730003B01019690933B0180933A0180913A01ED
:1007400090913B018031910540F38DE391E0998BCD
:10075000888BE3E1F1E0FB8BEA8BF8E0FC8BEA8924
:10076000FB8900802A893B892F5F3F4F3B8B2A8B77
:10077000E889F9890082288939892F5F3F4F398BB1
:10078000288B3C8931503C8B8C89882341F710920F
:100790003B0110923A011CC080913A0190913B01BB
:1007A000FC01E35CFE4F8081882349F480913A018B
:1007B00090913B01FC01E35CFE4F80E280838091DD
:1007C0003A0190913B01019690933B0180933A014D
:1007D00080913A0190913B0180319105E8F21092AD
:1007E0003B0110923A0113C080913A0190913B0174
:1007F000FC01E35CFE4F80810E941E0180913A0162
:1008000090913B01019690933B0180933A01809136
:100810003A0190913B018031910530F31092010132
:100820001092000181E080933401E9E3F0E08081DF
:100830009927847090701F821E82009721F4E1E056
:10084000F0E0FF83EE8380910001909101012E8101
:100850003F812823392380913501909136018223ED
:100860009323009709F488C06EC080E69AEE9093B7
:100870003B0180933A0109C080913A0190913B017C
:10088000019790933B0180933A0180913A019091B6
:100890003B01009789F780913D01809339011092C7
:1008A0003B0110923A011AC020913A0130913B016C
:1008B00080913A0190913B010196FC01E35CFE4F6F
:1008C0008081F901E35CFE4F808380913A01909131
:1008D0003B01019690933B0180933A0180913A014C
:1008E00090913B018F309105F8F28091390180930E
:1008F0004C0180913401813021F480E80E94D700BE
:1009000003C080EC0E94D70010923B0110923A0184
:1009100013C080913A0190913B01FC01E35CFE4FD2
:1009200080810E941E0180913A0190913B010196C5
:1009300090933B0180933A0180913A0190913B0161
:100940008031910530F3E9E3F0E0808199278470EC
:1009500090701D82009711F4F1E0FD8380913401C5
:100960008D8B2D89222311F031E03D8B8D899D8166
:100970008923882309F079CFE9E3F0E08081992782
:10098000887090701C821B82009721F4E1E0F0E0F7
:10099000FC83EB8380910001909101012B813C81CC
:1009A00028233923809135019091360182239323A6
:1009B000009709F493C081E00E94D70080EC0E9468
:1009C000D70010923B0110923A0111C080913A0178
:1009D00090913B01FC01E35CFE4F108280913A0153
:1009E00090913B01019690933B0180933A01809155
:1009F0003A0190913B018031910540F32DE331E0C4
:100A00003F8B2E8B8BE191E0998F888F98E09A8FA6
:100A1000E88DF98D0080288D398D2F5F3F4F398FFC
:100A2000288FEE89FF8900822E893F892F5F3F4FF3
:100A30003F8B2E8B3A8D31503A8F8A8D882341F728
:100A400010923B0110923A011CC080913A019091A2
:100A50003B01FC01E35CFE4F8081882349F48091D7
:100A60003A0190913B01FC01E35CFE4F80E2808300
:100A700080913A0190913B01019690933B018093C4
:100A80003A0180913A0190913B0180319105E8F261
:100A900010923B0110923A0113C080913A0190915B
:100AA0003B01FC01E35CFE4F80810E941E018091AE
:100AB0003A0190913B01019690933B0180933A015A
:100AC00080913A0190913B018031910530F3109271
:100AD00001011092000182E080933401E9E3F0E02B
:100AE00080819927807190701A821982009721F471
:100AF000E1E0F0E0FA83E983809100019091010147
:100B000029813A812823392380913501909136013A
:100B100082239323009709F440C081E00E94D7000C
:100B200083E291E00E9463018EE190E090933B01AB
:100B300080933A011FC080E395E79093380180933A
:100B4000370109C080913701909138010197909346
:100B500038018093370180913701909138010097D7
:100B600089F780913A0190913B01019790933B0165
:100B700080933A0180913A0190913B010097D9F618
:100B8000109201011092000188E00E94D70010929B
:100B900036011092350110923401E9E3F0E08081D2
:100BA00099279C0121703070E9E3F0E0808199275A
:100BB00082709070282B392BE9E3F0E0808199272F
:100BC00084709070282B392BE9E3F0E0808199271D
:100BD00088709070282B392BE9E3F0E08081992709
:100BE00080719070822B932B8F31910509F02BCD62
:100BF00081E090E0909301018093000124CD97FB68
:100C0000092E07260AD077FD04D027D006D0002071
:100C10001AF4709561957F4F0895F6F79095819538
:100C20009F4F089597FB092E05260ED057FD04D03F
:100C300028D00AD0001C38F4509540953095219565
:100C40003F4F4F4F5F4F0895F6F790958095709501
:100C500061957F4F8F4F9F4F0895AA1BBB1B51E19A
:100C600007C0AA1FBB1FA617B70710F0A61BB70B1C
:100C7000881F991F5A95A9F780959095BC01CD01C1
:100C80000895A1E21A2EAA1BBB1BFD010DC0AA1FCD
:100C9000BB1FEE1FFF1FA217B307E407F50720F0E5
:100CA000A21BB30BE40BF50B661F771F881F991F60
:100CB0001A9469F760957095809590959B01AC01A9
:080CC000BD01CF010895FFCF33
:100CC80001002020202057656C636F6D652020206F
:100CD800202000436F6E666C75780052616D7061FC
:100CE800726400202020205475726E204F464620E2
:040CF8002020200098
:00000001FF
